:020000040000FA
:0A000000000000008FEF00F09DD01B
:08001800F1D00F6E960E066E8A
:10002000980E076E55D8D8B4CA90D8A4CA80FC0FD1
:10003000D8A0CA92D8B0CA82800E066E960E076EFD
:10004000980E0A6E0B6ACAB025D8CAB223D842D815
:100050000604CB6E06C008F007C009F000500C6E15
:100060000D6E003C0D6A4BD80B500F2E0AD0BE6EA1
:100070000C0EBD6E0ABEBD8A0ABCBD889394CA84AC
:100080001200BB6E0C0EBA6E0ABEBA8A0ABCBA88DF
:100090009492F5D700D8D8900A320732063212006F
:1000A000096A086EFF0E0826092200D0D8A01200A7
:1000B000030E076EE60E02D8F5D7076AFE0F066E2E
:1000C000E86A075AD8A012000000060600D0F8D748
:1000D0000B6A0A6A100EF36E07340A360B360850A4
:1000E0000A5C09500B5805E308500A5E09500B5A88
:1000F000D88006360736F32EEFD706501200085088
:100100000C02F3CF0AF0F4CF0BF009500C02F350BD
:100110000B2608500D02F3500B260A5012004F0E0A
:10012000AF6E240EAC6E900EAB6E0001C69A430EFD
:10013000926EE00E936EC00E946E0F0EC16E070E9F
:10014000B46E73D000019EAA1BD0060EAB1412E150
:10015000E2CF39F0E1CF38F03A2A11EE00F03A5010
:10016000E126000EE222AECFE7FF39C0E2FF38C041
:10017000E1FF1100AE50AE50AB98AB88110008D033
:10018000F2A406D0F294144A152AD66A817A110094
:1001900011003A503B5C14E03B2AEACF07F0E9CF6C
:1001A00006F001EE00F03B50E926000EEA22EF5087
:1001B000066E07C0EAFF06C0E9FFD880120004D02F
:1001C000E868066ED8A0120012003A6A3B6A9D8A5F
:1001D0009F8AF28EF28CF28A12009D9A01EE00F054
:1001E000010EF46EF36AF306000EF45AEE6AF45050
:1001F000F310F9E13A6A3B6A9D8A1200F29EE0CF61
:100200006EF7D8CF6FF7E8CF70F7F28E0001A192AA
:10021000F29E6EC7E0FF6FC7D8FF70C7E8FFF28E8F
:1002200010009EA8FED7AD6E120092988998939404
:100230008A94949A8B9A94988B9894968B9694948B
:100240008B9494928B9294908B90929A899A2E6A26
:100250002D6A306A2F6A326A316A346A336A366AC2
:10026000356A9294899492968996939A8A9A006AAA
:10027000260E096E280E086E020ECFDE006A260ECC
:10028000096E280E086E010EC8DE286A7BEC06F0A7
:1002900078EC08F0939A8A8A320E02DF939A8A9A4F
:1002A000266A93DF9ADFCD6AF294F28A870ED56EC2
:1002B000B16AA192A082D08EA292B00EB16E69DF17
:1002C000166EBE0E165C08E3FE0E165C03E36FEFBF
:1002D00003F002D0186A03D216AE21D0186A8D0E30
:1002E000165C05E116C018F019681A6817D09D0E43
:1002F000165C05E116C018F01B681C680FD0AD0E27
:10030000165C05E116C018F01D681E6807D0BD0E0A
:10031000165C04E116C018F01F682068E0D118527E
:1003200002E1DDD1DCD18D0E185CD8A440D01928B3
:1003300003E116C019F039D03D0E195C04E1269096
:100340008B9A2C9031D03E0E195C04E126928B984A
:100350002C922AD03F0E195C04E126948B962C94A3
:1003600023D0400E195C04E126968B902C961CD06D
:10037000420E195C04E12698899A2C9815D07E0EBD
:10038000195C08E1006A260E096E280E086E010E3F
:1003900044DE0AD07F0E195C07E1006A260E096E62
:1003A000280E086E020E39DE196899D198D19D0E7B
:1003B000185CD8A479D11B2803E116C01BF072D1B8
:1003C00016C01CF01C523BE13D0E1B5C04E1269064
:1003D0008B9A2C9032D03E0E1B5C04E126928B98B7
:1003E0002C922BD03F0E1B5C04E126948B962C9410
:1003F00024D0400E1B5C04E126968B902C961DD0D9
:10040000420E1B5C04E12698899A2C9816D07E0E29
:100410001B5C08E1006A260E096E280E086E010EAC
:10042000FCDD0BD07F0E1B5C08E1006A260E096E16
:10043000280E086E020E0DEC00F01B6850D13D0E28
:100440001B5C34E12D5202E12E52D8A42C80000115
:100450002680D7CF13F0D6CF12F002EE6EF0D890F0
:100460001C34E926000EEA22EECF01F0EFCF02F0B5
:1004700002C03DF001C03CF03CC001F03DC002F0C4
:1004800001501224226E02501320236E000E1420FD
:10049000246E000E1520256E25C047F024C046F0BE
:1004A00023C051F022C050F08B8AFBD03E0E1B5C63
:1004B00034E12F5202E13052D8A42C82000126826E
:1004C000D7CF13F0D6CF12F003EE6EF0D8901C34D5
:1004D000E926000EEA22EECF01F0EFCF02F002C0D3
:1004E0003FF001C03EF03EC001F03FC002F00150BD
:1004F0001224226E02501320236E000E1420246E4C
:10050000000E1520256E25C049F024C048F023C0F8
:1005100053F022C052F08B88C4D03F0E1B5C34E1F4
:10052000315202E13252D8A42C8400012684D7CF64
:1005300013F0D6CF12F004EE6EF0D8901C34E926FA
:10054000000EEA22EECF01F0EFCF02F002C041F040
:1005500001C040F040C001F041C002F0015012243F
:10056000226E02501320236E000E1420246E000E03
:100570001520256E25C04BF024C04AF023C055F04D
:1005800022C054F08B868DD0400E1B5C34E1335278
:1005900002E13452D8A42C8600012686D7CF13F06E
:1005A000D6CF12F005EE6EF0D8901C34E926000E7E
:1005B000EA22EECF01F0EFCF02F002C043F001C01B
:1005C00042F042C001F043C002F001501224226EFA
:1005D00002501320236E000E1420246E000E1520EE
:1005E000256E25C04DF024C04CF023C057F022C02A
:1005F00056F08B8056D0420E1B5C34E1355202E13E
:100600003652D8A42C8800012688D7CF13F0D6CF35
:1006100012F006EE6EF0D8901C34E926000EEA22A5
:10062000EECF01F0EFCF02F002C045F001C044F080
:1006300044C001F045C002F001501224226E025065
:100640001320236E000E1420246E000E1520256E3C
:1006500025C04FF024C04EF023C059F022C058F0FE
:10066000898A1FD07E0E1B5C0DE1D8901C34376E3A
:1006700037C000F0260E096E280E086E010E0DEC34
:1006800000F00FD07F0E1B5C0CE1D8901C34376E4D
:1006900037C000F0260E096E280E086E020E0DEC13
:1006A00000F01B681CD01BD0AD0E185C0BE11D28A0
:1006B00003E116C01DF004D016C01EF09AEC05F040
:1006C0000ED00DD0BD0E185C0AE11F2803E116C044
:1006D0001FF004D016C020F0FFEC05F000D026A0DB
:1006E00039D046C024F047C025F050C022F051C098
:1006F00023F0D7CF13F0D6CF12F02250125C235044
:100700001358245014582550155823E38B9A2690DB
:100710002CA01FD02D5202E12E521AE0D7CF13F099
:10072000D6CF12F02D501224226E2E501320236E9D
:10073000000E1420246E000E1520256E25C05BF0DF
:1007400024C05AF023C065F022C064F0000101D03B
:100750002C9031D02CA02FD05AC024F05BC025F0B3
:1007600064C022F065C023F0D7CF13F0D6CF12F0CB
:100770002250125C235013582450145825501558F9
:100780001AE326803CC001F03DC002F00150122463
:10079000226E02501320236E000E1420246E000ED1
:1007A0001520256E25C047F024C046F023C051F027
:1007B00022C050F08B8A26A239D048C024F049C00C
:1007C00025F052C022F053C023F0D7CF13F0D6CF7C
:1007D00012F02250125C2350135824501458255004
:1007E000155823E38B9826922CA21FD02F5202E19A
:1007F00030521AE0D7CF13F0D6CF12F02F50122478
:10080000226E30501320236E000E1420246E000E32
:100810001520256E25C05DF024C05CF023C067F074
:1008200022C066F0000101D02C9231D02CA22FD032
:100830005CC024F05DC025F066C022F067C023F0E4
:10084000D7CF13F0D6CF12F02250125C235013589A
:1008500024501458255015581AE326823EC001F042
:100860003FC002F001501224226E02501320236E6A
:10087000000E1420246E000E1520256E25C049F0B0
:1008800024C048F023C053F022C052F08B8826A425
:1008900039D04AC024F04BC025F054C022F055C0D6
:1008A00023F0D7CF13F0D6CF12F02250125C235092
:1008B0001358245014582550155823E38B9626942A
:1008C0002CA41FD0315202E132521AE0D7CF13F0DC
:1008D000D6CF12F031501224226E32501320236EE4
:1008E000000E1420246E000E1520256E25C05FF02A
:1008F00024C05EF023C069F022C068F0000101D07E
:100900002C9431D02CA42FD05EC024F05FC025F0F1
:1009100068C022F069C023F0D7CF13F0D6CF12F011
:100920002250125C23501358245014582550155847
:100930001AE3268440C001F041C002F001501224A5
:10094000226E02501320236E000E1420246E000E1F
:100950001520256E25C04BF024C04AF023C055F069
:1009600022C054F08B8626A639D04CC024F04DC04E
:1009700025F056C022F057C023F0D7CF13F0D6CFC2
:1009800012F02250125C2350135824501458255052
:10099000155823E38B9026962CA61FD0335202E1E4
:1009A00034521AE0D7CF13F0D6CF12F033501224BE
:1009B000226E34501320236E000E1420246E000E7D
:1009C0001520256E25C061F024C060F023C06BF0B7
:1009D00022C06AF0000101D02C9631D02CA62FD075
:1009E00060C024F061C025F06AC022F06BC023F023
:1009F000D7CF13F0D6CF12F02250125C23501358E9
:100A000024501458255015581AE3268642C001F088
:100A100043C002F001501224226E02501320236EB4
:100A2000000E1420246E000E1520256E25C04DF0FA
:100A300024C04CF023C057F022C056F08B8026A86B
:100A400039D04EC024F04FC025F058C022F059C014
:100A500023F0D7CF13F0D6CF12F02250125C2350E0
:100A60001358245014582550155823E3899A269872
:100A70002CA81FD0355202E136521AE0D7CF13F01E
:100A8000D6CF12F035501224226E36501320236E2A
:100A9000000E1420246E000E1520256E25C063F074
:100AA00024C062F023C06DF022C06CF0000101D0C0
:100AB0002C9831D02CA82FD062C024F063C025F030
:100AC0006CC022F06DC023F0D7CF13F0D6CF12F058
:100AD0002250125C23501358245014582550155896
:100AE0001AE3268844C001F045C002F001501224E8
:100AF000226E02501320236E000E1420246E000E6E
:100B00001520256E25C04FF024C04EF023C059F0AB
:100B100022C058F0898A26502C24016E026A0236BF
:100B20000250011005E1010E155C02E3156A146A1A
:100B30005FEF01F03D0E1D5C11E11E520CE000EE76
:100B40006EF0D8901E34E926000EEA22EECF2DF08A
:100B5000EFCF2EF002D02E6A2D6A4FD03E0E1D5CD4
:100B600011E11E520CE000EE6EF0D8901E34E92622
:100B7000000EEA22EECF2FF0EFCF30F002D0306A35
:100B80002F6A3BD03F0E1D5C11E11E520CE000EEBF
:100B90006EF0D8901E34E926000EEA22EECF31F036
:100BA000EFCF32F002D0326A316A27D0400E1D5C9E
:100BB00011E11E520CE000EE6EF0D8901E34E926D2
:100BC000000EEA22EECF33F0EFCF34F002D0346AD9
:100BD000336A13D0420E1D5C10E11E520CE000EE91
:100BE0006EF0D8901E34E926000EEA22EECF35F0E2
:100BF000EFCF36F002D0366A356A1D681200420E19
:100C00001F5C09E1205203E124D8286A03D08988B7
:100C100020C028F004D07B0E1F5CD8B402D81F6817
:100C20001200266A2C6A006A260E096E280E086ECB
:100C3000010E0DEC00F0006A260E096E280E086EFB
:100C4000020E0DEC00F08B9A8B988B968B90899A04
:100C50001200266A2C6A8998006A260E096E280EF0
:100C6000086E010E0DEC00F0006A260E096E280ECB
:100C7000086E020E0DEC00F08B9A8B988B968B9081
:100C8000899A2E6A2D6A306A2F6A326A316A346A0A
:100C9000336A366A356A1200C9EC00F0166EBE0E71
:100CA000165C04E3FE0E165C01E2186A16AE09D06B
:100CB000186ABD0E165C04E116C018F01F682068A3
:100CC00014D0BD0E185C11E11F2803E116C01FF0FF
:100CD0000CD016C028F0420E1F5C07E11F68285296
:100CE00004E089888A845FEF01F0010E155C02E35D
:100CF000156A146AD1D7A20E716EC30E706E980E6B
:100D0000736E990E726E930E756EC20E746E8F0EA8
:100D1000776E120E766E8A0E796E880E786E860E5B
:100D20007B6E230E7A6E810E7D6EE10E7C6E7D0EE3
:100D30007F6EC30E7E6E790E816FC50E806F750E4D
:100D4000836FE80E826F720E856F2B0E846F6E0EAE
:100D5000876F8B0E866F6B0E896F0A0E886F670E1A
:100D60008B6FA40E8A6F640E8D6F5B0E8C6F610E9D
:100D70008F6F2C0E8E6F5E0E916F160E906F5B0E46
:100D8000936F1A0E926F580E956F360E946F550E24
:100D9000976F6A0E966F520E996FB40E986F500E41
:100DA0009B6F150E9A6F4D0E9D6F8A0E9C6F4B0EAA
:100DB0009F6F140E9E6F480EA16FB30EA06F460E6C
:100DC000A36F640EA26F440EA56F290EA46F410E8F
:100DD000A76FA6693F0EA96FE70EA86F3D0EAB6F18
:100DE000E00EAA6F3B0EAD6FEA0EAC6F3A0EAF6F1E
:100DF000030EAE6F380EB16F2C0EB06F360EB36FA0
:100E0000640EB26F340EB56FAA0EB46F320EB76FA8
:100E1000FE0EB66F310EB96F600EB86F2F0EBB6F3E
:100E2000CF0EBA6F2E0EBD6F4B0EBC6F2C0EBF6F68
:100E3000D30EBE6F2B0EC16F670EC06F2A0EC36F2D
:100E4000060EC26F280EC56FB10EC46F270EC76F96
:100E5000660EC66F260EC96FC86F240ECB6FF10EDB
:100E6000CA6F230ECD6FC50ECC6F220ECF6FA20EB0
:100E7000CE6F210ED16F890ED06F200ED36F790EF9
:100E8000D26F1F0ED56F710ED46F1E0ED76F710EFD
:100E9000D66F1D0ED96F7A0ED86F1C0EDB6F8B0EBE
:100EA000DA6F1B0EDD6FA30EDC6F1A0EDF6FC30E41
:100EB000DE6F190EE16FE90EE06F190EE36F170E8A
:100EC000E26F180EE56F4B0EE46F170EE76F860E9C
:100ED000E66F160EE96FC70EE86F160EEB6F0E0E7B
:100EE000EA6F150EED6F5B0EEC6F140EEF6FAD0E2B
:100EF000EE6F140EF16F050EF06F130EF36F630EAD
:100F0000F26F120EF56FC50EF46F120EF76F2D0E05
:100F1000F66F110EF96F990EF86F110EFB6F0A0E36
:100F2000FA6F100EFD6F800EFC6F0F0EFF6FFA0E42
:100F3000FE6F0F0E0101016F780E006F0E0E036F32
:100F4000FA0E026F0E0E056F810E046F0E0E076F04
:100F50000B0E066F0D0E096F990E086F0D0E0B6FBD
:100F60002B0E0A6F0C0E0D6FC00E0C6F0C0E0F6F58
:100F7000580E0E6F0B0E116FF40E106F0B0E136FD9
:100F8000930E126F0B0E156F350E146F0A0E176F3E
:100F9000DA0E166F0A0E196F820E186F0A0E1B6F8B
:100FA0002C0E1A6F090E1D6FDA0E1C6F090E1F6FC3
:100FB0008A0E1E6F090E216F3C0E206F080E236FE4
:100FC000F10E226F080E256FA90E246F080E276FF1
:100FD000620E266F080E296F1E0E286F070E2B6FEC
:100FE000DC0E2A6F070E2D6F9C0E2C6F070E2F6FD5
:100FF0005F0E2E6F070E316F230E306F060E336FAC
:10100000E90E326F060E356FB10E346F060E376F74
:101010007A0E366F060E396F460E386F060E3B6F2E
:10102000130E3A6F050E3D6FE10E3C6F050E3F6FDC
:10103000B20E3E6F050E416F830E406F050E436F7B
:10104000570E426F050E456F2B0E446F050E476F0E
:10105000010E466F040E496FD90E486F040E4B6F98
:10106000B10E4A6F040E4D6F8B0E4C6F040E4F6F16
:10107000660E4E6F040E516F430E506F040E536F89
:10108000200E526F030E556FFE0E546F030E576FF6
:10109000DE0E566F030E596FBF0E586F030E5B6F57
:1010A000A00E5A6F030E5D6F830E5C6F030E5F6FB1
:1010B000660E5E6F030E616F4B0E606F030E636F03
:1010C000300E626F030E656F160E646F020E676F4F
:1010D000FD0E666F020E696FE50E686F020E6B6F94
:1010E000CD0E6A6F020E6D6FB60E6C6F00011200AE
:1010F0000101716B2A0E706F020E176E0001800ED7
:10110000175C20E21704056E01EE6EF0D8900534EE
:10111000E926000EEA22EECF03F0EFCF04F0050E31
:101120000324016E000E0420026E01EE6EF0D890D2
:101130001734E926000EEA2201C0EEFF02C0EFFFDD
:10114000172ADCE30201716BB80E706F736BBA0E75
:10115000726F756BBB0E746F776BBC0E766F796BAD
:10116000BD0E786F7B6BBE0E7A6F7D6BBF0E7C6F92
:101170007F6BC10E7E6F816BC20E806F836BC30E5F
:10118000826F856BC40E846F876BC50E866F896B0B
:10119000C60E886F8B6BC80E8A6F8D6BC90E8C6FF5
:1011A0008F6BCA0E8E6F916BCB0E906F936BCC0EC4
:1011B000926F956BCD0E946F976BCF0E966F996B68
:1011C000D00E986F9B6BD10E9A6F9D6BD20E9C6F59
:1011D0009F6BD30E9E6FA16BD40EA06FA36BD60E28
:1011E000A26FA56BD70EA46FA76BD80EA66FA96BC5
:1011F000D90EA86FAB6BDA0EAA6FAD6BDB0EAC6FBE
:10120000AF6BDC0EAE6FB16BDE0EB06FB36BDF0E8B
:10121000B26FB56BE00EB46FB76BE10EB66FB96B22
:10122000E20EB86FBB6BE30EBA6FBD6BE50EBC6F21
:10123000BF6BE60EBE6FC16BE70EC06FC36BE80EEF
:10124000C26FC56BE90EC46FC76BEA0EC66FC96B80
:10125000EC0EC86FCB6BED0ECA6FCD6BEE0ECC6F84
:10126000CF6BEF0ECE6FD16BF00ED06FD36BF10E54
:10127000D26FD56BF30ED46FD76BF40ED66FD96BDC
:10128000F50ED86FDB6BF60EDA6FDD6BF70EDC6FE9
:10129000DF6BF80EDE6FE16BF90EE06FE36BFB0EB8
:1012A000E26FE56BFC0EE46FE76BFD0EE66FE96B3A
:1012B000FE0EE86FEB6BEA69010EED6FEC6BEF6F02
:1012C000020EEE6F010EF16F030EF06F010EF36F61
:1012D000040EF26F010EF56F050EF46F010EF76F3D
:1012E000060EF66F010EF96F070EF86F010EFB6F19
:1012F000090EFA6F010EFD6F0A0EFC6F010EFF6FF3
:101300000B0EFE6F010E0301016F0C0E006F010E3C
:10131000036F0D0E026F010E056F0E0E046F010EAE
:10132000076F100E066F010E096F110E086F010E88
:101330000B6F120E0A6F010E0D6F130E0C6F010E64
:101340000F6F140E0E6F010E116F150E106F010E40
:10135000136F170E126F010E156F180E146F010E1A
:10136000176F190E166F010E196F1A0E186F010EF6
:101370001B6F1B0E1A6F010E1D6F1C0E1C6F010ED2
:101380001F6F1D0E1E6F010E216F1F0E206F010EAD
:10139000236F200E226F010E256F210E246F010E88
:1013A000276F220E266F010E296F230E286F010E64
:1013B0002B6F240E2A6F010E2D6F260E2C6F010E3F
:1013C0002F6F270E2E6F010E316F280E306F010E1A
:1013D000336F290E326F010E356F2A0E346F010EF6
:1013E000376F2B0E366F010E396F2D0E386F010ED1
:1013F0003B6F2E0E3A6F010E3D6F2F0E3C6F010EAC
:101400003F6F300E3E6F010E416F310E406F010E87
:10141000436F320E426F010E456F340E446F010E62
:10142000476F350E466F010E496F360E486F010E3D
:101430004B6F370E4A6F010E4D6F380E4C6F010E19
:101440004F6F390E4E6F010E516F3A0E506F010EF5
:10145000536F3C0E526F010E556F3D0E546F010ECF
:10146000576F3E0E566F010E596F3F0E586F010EAB
:101470005B6F400E5A6F010E5D6F410E5C6F010E87
:101480005F6F430E5E6F010E616F440E606F010E61
:10149000636F450E626F010E656F460E646F010E3D
:1014A000676F470E666F010E696F480E686F010E19
:1014B0006B6F4A0E6A6F010E6D6F4B0E6C6F716B26
:1014C0002F0E706F736B340E726F756B390E746FF5
:1014D000776B3E0E766F796B420E786F7B6B470EA3
:1014E0007A6F7D6B4C0E7C6F7F6B510E7E6F816BC4
:1014F000560E806F836B5B0E826F856B600E846F00
:10150000876B650E866F896B690E886F8B6B6E0EAD
:101510008A6F8D6B730E8C6F8F6B780E8E6F916BE5
:101520007D0E906F936B820E926F956B870E946F0A
:10153000976B8C0E966F996B900E986F9B6B950EB8
:101540009A6F9D6B9A0E9C6F9F6B9F0E9E6FA16B07
:10155000A40EA06FA36BA90EA26FA56BAE0EA46F15
:10156000A76BB30EA66FA96BB70EA86FAB6BBC0EC3
:10157000AA6FAD6BC10EAC6FAF6BC60EAE6FB16B29
:10158000CB0EB06FB36BD00EB26FB56BD50EB46F20
:10159000B76BDA0EB66FB96BDE0EB86FBB6BE30ECE
:1015A000BA6FBD6BE80EBC6FBF6BED0EBE6FC16B4B
:1015B000F20EC06FC36BF70EC26FC56BFC0EC46F2B
:1015C000010EC76FC66FC96F050EC86F010ECB6FD6
:1015D0000A0ECA6F010ECD6F0F0ECC6F010ECF6FCA
:1015E000140ECE6F010ED16F190ED06F010ED36F96
:1015F0001E0ED26F010ED56F230ED46F010ED76F62
:10160000280ED66F010ED96F2C0ED86F010EDB6F2E
:10161000310EDA6F010EDD6F360EDC6F010EDF6FFB
:101620003B0EDE6F010EE16F400EE06F010EE36FC7
:10163000450EE26F010EE56F4A0EE46F010EE76F93
:101640004F0EE66F010EE96F530EE86F010EEB6F60
:10165000580EEA6F010EED6F5D0EEC6F010EEF6F2D
:10166000620EEE6F010EF16F670EF06F010EF36FF9
:101670006C0EF26F010EF56F710EF46F010EF76FC5
:10168000760EF66F010EF96F7A0EF86F010EFB6F92
:101690007F0EFA6F010EFD6F840EFC6F010EFF6F5F
:1016A000890EFE6F010E0401016F8E0E006F010E98
:1016B000036F930E026F010E056F980E046F010EFB
:1016C000076F9D0E066F010E096FA10E086F010EC8
:1016D0000B6FA60E0A6F010E0D6FAB0E0C6F010E95
:1016E0000F6FB00E0E6F010E116FB50E106F010E61
:1016F000136FBA0E126F010E156FBF0E146F010E2D
:10170000176FC40E166F010E196FC80E186F010EF9
:101710001B6FCD0E1A6F010E1D6FD20E1C6F010EC6
:101720001F6FD70E1E6F010E216FDC0E206F010E92
:10173000236FE10E226F010E256FE60E246F010E5E
:10174000276FEB0E266F010E296FEF0E286F010E2B
:101750002B6FF40E2A6F010E2D6FF90E2C6F010EF8
:101760002F6FFE0E2E6F020E316F030E306F020EC2
:10177000336F080E326F020E356F0D0E346F020E8E
:10178000376F120E366F020E396F160E386F020E5B
:101790003B6F1B0E3A6F020E3D6F200E3C6F020E28
:1017A0003F6F250E3E6F020E416F2A0E406F020EF4
:1017B000436F2F0E426F020E456F340E446F020EC0
:1017C000476F390E466F020E496F3D0E486F020E8D
:1017D0004B6F420E4A6F020E4D6F470E4C6F020E5A
:1017E0004F6F4C0E4E6F020E516F510E506F020E26
:1017F000536F560E526F020E556F5B0E546F020EF2
:10180000576F600E566F020E596F640E586F020EBE
:101810005B6F690E5A6F020E5D6F6E0E5C6F020E8B
:101820005F6F730E5E6F020E616F780E606F020E57
:10183000636F7D0E626F020E656F820E646F020E23
:10184000676F870E666F020E696F8B0E686F020EF0
:101850006B6F900E6A6F020E6D6F950E6C6F716BF1
:101860002F0E706F736B340E726F756B390E746F51
:10187000776B3E0E766F796B420E786F7B6B470EFF
:101880007A6F7D6B4C0E7C6F7F6B510E7E6F816B20
:10189000560E806F836B5B0E826F856B600E846F5C
:1018A000876B650E866F896B690E886F8B6B6E0E0A
:1018B0008A6F8D6B730E8C6F8F6B780E8E6F916B42
:1018C0007D0E906F936B820E926F956B870E946F67
:1018D000976B8C0E966F996B900E986F9B6B950E15
:1018E0009A6F9D6B9A0E9C6F9F6B9F0E9E6FA16B64
:1018F000A40EA06FA36BA90EA26FA56BAE0EA46F72
:10190000A76BB30EA66FA96BB70EA86FAB6BBC0E1F
:10191000AA6FAD6BC10EAC6FAF6BC60EAE6FB16B85
:10192000CB0EB06FB36BD00EB26FB56BD50EB46F7C
:10193000B76BDA0EB66FB96BDE0EB86FBB6BE30E2A
:10194000BA6FBD6BE80EBC6FBF6BED0EBE6FC16BA7
:10195000F20EC06FC36BF70EC26FC56BFC0EC46F87
:10196000010EC76FC66FC96F050EC86F010ECB6F32
:101970000A0ECA6F010ECD6F0F0ECC6F010ECF6F26
:10198000140ECE6F010ED16F190ED06F010ED36FF2
:101990001E0ED26F010ED56F230ED46F010ED76FBE
:1019A000280ED66F010ED96F2C0ED86F010EDB6F8B
:1019B000310EDA6F010EDD6F360EDC6F010EDF6F58
:1019C0003B0EDE6F010EE16F400EE06F010EE36F24
:1019D000450EE26F010EE56F4A0EE46F010EE76FF0
:1019E0004F0EE66F010EE96F530EE86F010EEB6FBD
:1019F000580EEA6F010EED6F5D0EEC6F010EEF6F8A
:101A0000620EEE6F010EF16F670EF06F010EF36F55
:101A10006C0EF26F010EF56F710EF46F010EF76F21
:101A2000760EF66F010EF96F7A0EF86F010EFB6FEE
:101A30007F0EFA6F010EFD6F840EFC6F010EFF6FBB
:101A4000890EFE6F010E0501016F8E0E006F010EF3
:101A5000036F930E026F010E056F980E046F010E57
:101A6000076F9D0E066F010E096FA10E086F010E24
:101A70000B6FA60E0A6F010E0D6FAB0E0C6F010EF1
:101A80000F6FB00E0E6F010E116FB50E106F010EBD
:101A9000136FBA0E126F010E156FBF0E146F010E89
:101AA000176FC40E166F010E196FC80E186F010E56
:101AB0001B6FCD0E1A6F010E1D6FD20E1C6F010E23
:101AC0001F6FD70E1E6F010E216FDC0E206F010EEF
:101AD000236FE10E226F010E256FE60E246F010EBB
:101AE000276FEB0E266F010E296FEF0E286F010E88
:101AF0002B6FF40E2A6F010E2D6FF90E2C6F010E55
:101B00002F6FFE0E2E6F020E316F030E306F020E1E
:101B1000336F080E326F020E356F0D0E346F020EEA
:101B2000376F120E366F020E396F160E386F020EB7
:101B30003B6F1B0E3A6F020E3D6F200E3C6F020E84
:101B40003F6F250E3E6F020E416F2A0E406F020E50
:101B5000436F2F0E426F020E456F340E446F020E1C
:101B6000476F390E466F020E496F3D0E486F020EE9
:101B70004B6F420E4A6F020E4D6F470E4C6F020EB6
:101B80004F6F4C0E4E6F020E516F510E506F020E82
:101B9000536F560E526F020E556F5B0E546F020E4E
:101BA000576F600E566F020E596F640E586F020E1B
:101BB0005B6F690E5A6F020E5D6F6E0E5C6F020EE8
:101BC0005F6F730E5E6F020E616F780E606F020EB4
:101BD000636F7D0E626F020E656F820E646F020E80
:101BE000676F870E666F020E696F8B0E686F020E4D
:101BF0006B6F900E6A6F020E6D6F950E6C6F716B4E
:101C0000510E706F736B530E726F756B550E746F50
:101C1000776B570E766F796B580E786F7B6B5A0E19
:101C20007A6F7D6B5C0E7C6F7F6B5E0E7E6F816B5F
:101C3000600E806F836B610E826F856B630E846FA5
:101C4000876B650E866F896B670E886F8B6B680E6E
:101C50008A6F8D6B6A0E8C6F8F6B6C0E8E6F916BB3
:101C60006E0E906F936B700E926F956B710E946FFA
:101C7000976B730E966F996B750E986F9B6B770EC3
:101C80009A6F9D6B780E9C6F9F6B7A0E9E6FA16B07
:101C90007C0EA06FA36B7E0EA26FA56B800EA46F4F
:101CA000A76B810EA66FA96B830EA86FAB6B850E19
:101CB000AA6FAD6B870EAC6FAF6B880EAE6FB16B5A
:101CC0008A0EB06FB36B8C0EB26FB56B8E0EB46FA5
:101CD000B76B900EB66FB96B910EB86FBB6B930E6E
:101CE000BA6FBD6B950EBC6FBF6B970EBE6FC16BAD
:101CF000980EC06FC36B9A0EC26FC56B9C0EC46FFB
:101D0000C76B9E0EC66FC96BA00EC86FCB6BA10EC2
:101D1000CA6FCD6BA30ECC6FCF6BA50ECE6FD16B00
:101D2000A70ED06FD36BA90ED26FD56BAA0ED46F4E
:101D3000D76BAC0ED66FD96BAE0ED86FDB6BB00E17
:101D4000DA6FDD6BB10EDC6FDF6BB30EDE6FE16B54
:101D5000B50EE06FE36BB70EE26FE56BB90EE46FA3
:101D6000E76BBA0EE66FE96BBC0EE86FEB6BBE0E6D
:101D7000EA6FED6BC00EEC6FEF6BC10EEE6FF16BA7
:101D8000C30EF06FF36BC50EF26FF56BC70EF46FF9
:101D9000F76BC90EF66FF96BCA0EF86FFB6BCC0EC2
:101DA000FA6FFD6BCE0EFC6FFF6BD00EFE6F06015F
:101DB000016BD10E006F036BD30E026F056BD50E56
:101DC000046F076BD70E066F096BD90E086F0B6B8C
:101DD000DA0E0A6F0D6BDC0E0C6F0F6BDE0E0E6FE2
:101DE000116BE00E106F136BE10E126F156BE30EAB
:101DF000146F176BE50E166F196BE70E186F1B6BE0
:101E0000E90E1A6F1D6BEA0E1C6F1F6BEC0E1E6F36
:101E1000216BEE0E206F236BF00E226F256BF10EFF
:101E2000246F276BF30E266F296BF50E286F2B6B33
:101E3000F70E2A6F2D6BF90E2C6F2F6BFA0E2E6F8B
:101E4000316BFC0E306F336BFE0E326F010E356F4F
:101E5000346B376F366F396F030E386F010E3B6F7F
:101E6000050E3A6F010E3D6F070E3C6F010E3F6F7E
:101E7000090E3E6F010E416F0A0E406F010E436F57
:101E80000C0E426F010E456F0E0E446F010E476F30
:101E9000100E466F010E496F120E486F010E4B6F08
:101EA000130E4A6F010E4D6F150E4C6F010E4F6FE2
:101EB000170E4E6F010E516F190E506F010E536FBA
:101EC0001A0E526F010E556F1C0E546F010E576F94
:101ED0001E0E566F010E596F200E586F010E5B6F6C
:101EE000220E5A6F010E5D6F230E5C6F010E5F6F45
:101EF000250E5E6F010E616F270E606F010E636F1E
:101F0000290E626F010E656F2A0E646F010E676FF6
:101F10002C0E666F010E696F2E0E686F010E6B6FCF
:101F2000300E6A6F010E6D6F320E6C6F716B2F0E7B
:101F3000706F736B340E726F756B390E746F776BD5
:101F40003E0E766F796B420E786F7B6B470E7A6F21
:101F50007D6B4C0E7C6F7F6B510E7E6F816B560ECE
:101F6000806F836B5B0E826F856B600E846F876BF7
:101F7000650E866F896B690E886F8B6B6E0E8A6F2C
:101F80008D6B730E8C6F8F6B780E8E6F916B7D0ED9
:101F9000906F936B820E926F956B870E946F976B19
:101FA0008C0E966F996B900E986F9B6B950E9A6F37
:101FB0009D6B9A0E9C6F9F6B9F0E9E6FA16BA40EE4
:101FC000A06FA36BA90EA26FA56BAE0EA46FA76B3B
:101FD000B30EA66FA96BB70EA86FAB6BBC0EAA6F42
:101FE000AD6BC10EAC6FAF6BC60EAE6FB16BCB0EEF
:101FF000B06FB36BD00EB26FB56BD50EB46FB76B5D
:10200000DA0EB66FB96BDE0EB86FBB6BE30EBA6F4C
:10201000BD6BE80EBC6FBF6BED0EBE6FC16BF20EF9
:10202000C06FC36BF70EC26FC56BFC0EC46F010EA1
:10203000C76FC66FC96F050EC86F010ECB6F0A0E52
:10204000CA6F010ECD6F0F0ECC6F010ECF6F140E45
:10205000CE6F010ED16F190ED06F010ED36F1E0E11
:10206000D26F010ED56F230ED46F010ED76F280EDD
:10207000D66F010ED96F2C0ED86F010EDB6F310EAB
:10208000DA6F010EDD6F360EDC6F010EDF6F3B0E77
:10209000DE6F010EE16F400EE06F010EE36F450E43
:1020A000E26F010EE56F4A0EE46F010EE76F4F0E0F
:1020B000E66F010EE96F530EE86F010EEB6F580EDD
:1020C000EA6F010EED6F5D0EEC6F010EEF6F620EA9
:1020D000EE6F010EF16F670EF06F010EF36F6C0E75
:1020E000F26F010EF56F710EF46F010EF76F760E41
:1020F000F66F010EF96F7A0EF86F010EFB6F7F0E0F
:10210000FA6F010EFD6F840EFC6F010EFF6F890EDA
:10211000FE6F010E0701016F8E0E006F010E036F3F
:10212000930E026F010E056F980E046F010E076F7C
:102130009D0E066F010E096FA10E086F010E0B6F49
:10214000A60E0A6F010E0D6FAB0E0C6F010E0F6F16
:10215000B00E0E6F010E116FB50E106F010E136FE2
:10216000BA0E126F010E156FBF0E146F010E176FAE
:10217000C40E166F010E196FC80E186F010E1B6F7B
:10218000CD0E1A6F010E1D6FD20E1C6F010E1F6F48
:10219000D70E1E6F010E216FDC0E206F010E236F14
:1021A000E10E226F010E256FE60E246F010E276FE0
:1021B000EB0E266F010E296FEF0E286F010E2B6FAD
:1021C000F40E2A6F010E2D6FF90E2C6F010E2F6F7A
:1021D000FE0E2E6F020E316F030E306F020E336F44
:1021E000080E326F020E356F0D0E346F020E376F10
:1021F000120E366F020E396F160E386F020E3B6FDD
:102200001B0E3A6F020E3D6F200E3C6F020E3F6FA9
:10221000250E3E6F020E416F2A0E406F020E436F75
:102220002F0E426F020E456F340E446F020E476F41
:10223000390E466F020E496F3D0E486F020E4B6F0E
:10224000420E4A6F020E4D6F470E4C6F020E4F6FDB
:102250004C0E4E6F020E516F510E506F020E536FA7
:10226000560E526F020E556F5B0E546F020E576F73
:10227000600E566F020E596F640E586F020E5B6F40
:10228000690E5A6F020E5D6F6E0E5C6F020E5F6F0D
:10229000730E5E6F020E616F780E606F020E636FD9
:1022A0007D0E626F020E656F820E646F020E676FA5
:1022B000870E666F020E696F8B0E686F020E6B6F72
:1022C000900E6A6F020E6D6F950E6C6F000112001A
:0222D000FFD736
:020000040030CA
:0300010006170ED1
:020005008580F4
:060008000FC00FE00F40E5
:00000001FF
